:100000000C943E000C9459000C945B000C94590025
:100010000C9459000C9459000C9459000C945900FC
:100020000C9459000C9459000C9459000C945900EC
:100030000C9459000C9459000C9459000C945900DC
:100040000C9459000C9459000C9459000C945900CC
:100050000C94590099089B089D08A008A308A308C0
:10006000A308A308A508A508A508A508A508A5082C
:10007000A508A508A508A508A508A80811241FBE5D
:10008000CFE5D4E0DEBFCDBF10E0A0E6B0E0E4EB0A
:10009000F1E102C005900D92A637B107D9F710E043
:1000A000A6E7B0E001C01D92AC3DB107E1F70C94AA
:1000B000CC000C9400001F920F920FB60F921124E7
:1000C0002F933F934F935F936F937F938F939F9360
:1000D000AF93BF93EF93FF938DE00E94E60180936F
:1000E000D7006FEF8DE00E9405020000FF91EF91B5
:1000F000BF91AF919F918F917F916F915F914F9140
:100100003F912F910F900FBE0F901F9018951F9346
:100110001ABA8FE487BB83EC84BB1FEF11BB1BBAF9
:100120008FE088BB83E485BB80E182BB80E88BBF26
:100130008CE085BF84E085BF88EE93E00E94BE011D
:10014000AF9AA8980E9489020E94E20480E690E09B
:100150000E94F0048EE00E94E60182958F70805D1F
:100160008093D7000E94E704AE988CE68DB9109278
:100170009300109292001092D3001092D20010922D
:100180007800109277001093D4001093D80084E187
:1001900080937B001F910895CFE5D4E0DEBFCDBFF3
:1001A0000E9487000E94F5026EE270E081E090E01C
:1001B0000E947A04C0E010927B008091920090919E
:1001C00093008130910579F0823091051CF4892BE0
:1001D00039F011C08230910549F0039751F00BC0FE
:1001E0000E94110508C00E947A0505C00E94CD0733
:1001F00002C00E947308CC2339F482E080939800F7
:10020000C0939900C1E007C082E08093980081E02C
:1002100080939900C0E0B49BFECF84E180937B0083
:10022000979860E270E087E990E00E940D048FEFFC
:100230008093D4008093D80040919900242F3327D5
:1002400025FF03C08EEF8093D40024FF05C080916A
:10025000D4008D7F8093D40023FF05C08091D4000B
:100260008B7F8093D40026FF05C08091D400877FC8
:100270008093D4009091A800892F86588A3420F466
:100280008091D4008F7E06C096509A3628F48091D3
:10029000D4008F7B8093D4009091A600892F865044
:1002A0008A3620F48091D4008F7D06C096589A3407
:1002B00028F48091D4008F778093D4002091A200FD
:1002C000203428F48091D8008E7F8093D8009091BC
:1002D000A000913C28F08091D800877F8093D800BF
:1002E000213C28F08091D8008D7F8093D8009034F5
:1002F00028F48091D8008B7F8093D800242F332757
:1003000022FF05C08091D8008F7E8093D80021FF06
:1003100005C08091D8008F7D8093D80080919D008A
:1003200081FF05C08091D8008F7B8093D80020FF8B
:1003300005C08091D8008F778093D80080919C0071
:10034000282F332721FF05C08091D800807D80931E
:10035000D80022FF0AC08091D4008D7F8093D40002
:100360008091D800807F8093D80023FF05C08091C2
:10037000D800807E8093D800979A1DCFCF93DF93CB
:10038000CDB7DEB721970FB6F894DEBF0FBECDBF55
:10039000AC0120E030E02817390778F41982898110
:1003A0008E3430F489818F5F898389818E34D0F3D4
:1003B0002F5F3F4F2417350788F321960FB6F89427
:1003C000DEBF0FBECDBFDF91CF910895982F8FEF85
:1003D0008ABBC098C1989BBBC39800000000000076
:1003E00000000000C39A0000C19A00000000000055
:1003F000000000001ABAC09AC198C298000089B3E0
:10040000C29A0000C19A992708959FEF9ABBC0989D
:10041000C1988BBBC39800000000000000000000E2
:10042000C39A0000C19A0000000000000000000014
:10043000C09AC1986BBBC3980000C39A0000C19AD0
:100440001ABA08959C01FB014115510559F18FEF2E
:100450008ABBC098C1982BBBC39800000000000065
:100460000000C39A0000C19A0000000000000000D4
:10047000415050408FEF4F3F5807A1F01ABAC09A31
:10048000C198C298000089B38193C29A0000C19AB2
:100490000000000000000000415050408FEF4F3F2F
:1004A000580761F708959C01FB014115510509F4B6
:1004B0002FC08FEF8ABBC098C1982BBBC398000098
:1004C0000000000000000000C39A0000C19A000074
:1004D0000000000000000000415050408FEF4F3FEF
:1004E0005807A9F0C09AC19881918BBB0000C398AE
:1004F0000000C39A0000C19A000000000000000044
:100500000000415050408FEF4F3F580759F71ABA3B
:100510000895AF92BF92CF92DF92EF92FF920F9326
:100520001F93CF93DF93CDB7DEB7C050D1400FB646
:10053000F894DEBF0FBECDBFAA24BB2430E1E32E6A
:10054000F12C6E010894C11CD11C87010C0D1D1DDE
:100550008E2D0E94E601F80180836E2D8E2D0E9463
:1005600005020894E11CF11CFFEFEF16F10449F3BA
:1005700044F320E1E22EF12C8E2D0E94E601992712
:100580008E159F0519F09FEFA92EB92E0894E11C36
:10059000F11C8FEFE816F10479F374F380E1E82E93
:1005A000F12C86010E0D1F1DF80161918F018E2D1A
:1005B0000E9405020894E11CF11CFFEFEF16F10404
:1005C00099F394F3C501C050DF4F0FB6F894DEBF26
:1005D0000FBECDBFDF91CF911F910F91FF90EF9094
:1005E000DF90CF90BF90AF9008951F93CF93DF938C
:1005F0006EEA8FE00E94050268E085E00E94050235
:1006000080ED97E00E94BE0160E085E00E94050257
:100610008FEF8093BB00C3E6D0E06FEF8DE00E94C8
:1006200005022197D7FFF9CF8DE00E94E601C82F80
:10063000DD27C6FF09C01092BB0061E386E00E947F
:1006400005028FEF9FEF55C060E08AE00E9405022F
:1006500060E58BE00E94050261E08CE00E940502EB
:1006600060EE8EE00E9405028C2F807809F511E083
:100670001093BB0068E085E00E94050280ED97E0E2
:100680000E94BE0161E285E00E9405026EEE8FE0ED
:100690000E940502612F88E00E940502C3E1D0E0BC
:1006A0006FEF8DE00E9405022197D7FFF9CF1BC0A5
:1006B00082E08093BB0068E085E00E94050280ED47
:1006C00097E00E94BE0165E0862F0E9405026EEA57
:1006D0008FE00E94050261E088E00E9405026FEF52
:1006E0008DE00E94050261E386E00E94050280E041
:1006F00090E0DF91CF911F910895CF93DF93EC01AC
:1007000048E050E0BE0180E190E00E94530260E1C9
:1007100081E00E94050268E082E00E94050260918B
:10072000940084E00E94050260ED83E00E940502CF
:1007300067E080E00E94050288EC90E00E94BE0124
:100740008DE00E94E60180FFFBCF83E00E94E6017E
:10075000982F282F332722FDD3CF80E020FD81E082
:1007600026FD826097FD84609927DF91CF910895DF
:100770000F931F93CF93DF938C01EB01C230D10510
:100780001CF480E090E044C0CE01029798012E5FF7
:100790003F4FAC01B90180E190E00E94530260E15B
:1007A00081E00E9405028C2F8250682F82E00E9417
:1007B00005026091940084E00E940502F8018181A5
:1007C0008061682F83E00E940502F80182818823FE
:1007D00011F467E001C067E480E00E94050288EC44
:1007E00090E00E94BE018DE00E94E60180FFFBCFF9
:1007F00083E00E94E601982F282F332722FDBECFE9
:1008000080E020FD81E026FD826097FD84609927CD
:10081000DF91CF911F910F910895BF92CF92DF92F8
:10082000EF92FF920F931F93CF93DF937C018B0185
:1008300077FF03C080E090E04EC060E181E00E945D
:100840000502602F82E00E9405026091940084E01E
:100850000E940502F70181818069682F83E00E9470
:100860000502C0E0D0E0F7018281882311F463E043
:1008700001C063E480E00E94050284E190E00E94F0
:10088000BE018DE00E94E60180FFFBCF83E00E9465
:10089000E601B82E992740E4C42ED12CC822D922D3
:1008A00086FF04C02196C230D105ECF2EC01C17084
:1008B000D07080FF06C0A801B70180E190E00E94DF
:1008C000220280E0CD2B09F081E0CD2809F0826082
:1008D000B7FC84609927DF91CF911F910F91FF9012
:1008E000EF90DF90CF90BF9008958093940080E0C8
:1008F00090E00895DF92EF92FF920F931F93CF93B2
:10090000DF93CDB7DEB728970FB6F894DEBF0FBEE2
:10091000CDBF6F32710509F43FC06033710524F417
:100920006E32710529F03CC06033710581F138C029
:100930007FEFE72EF72E109294000E94F5028C01B3
:10094000892B89F586E690E00E947D0380FF2BC00D
:100950001A8261E0D62EDB82B801CE0101960E9498
:100960000D0480FF20C082E0809394008EE690E02A
:100970000E947D0380FF17C01A82DB82B801CE017E
:1009800001960E940D0480FF0EC0888502C08091F0
:10099000BB00E82EFF2407C00E947D037C0103C03A
:1009A0005FEFE52EF52EC70128960FB6F894DEBF4F
:1009B0000FBECDBFDF91CF911F910F91FF90EF90B0
:1009C000DF90089588E18AB98FE289B908955D9B27
:1009D000FECF8CB908955F9BFECF8CB19927089507
:1009E000CF93DF93EC018881882331F089910E94B5
:1009F000E70488818823D1F7DF91CF910895000023
:100A00000000000000000197D1F7089584E090E015
:100A10000E94FF04949882E090E00E94FF04949A60
:100A20000895B499FECF80E590E00E94FF041092F3
:100A30007B00779BFECF84E190E00E94FF042FB102
:100A40002093DB0080917B00992781309105D9F0BC
:100A5000823091051CF4892B39F02EC0823091052B
:100A6000A1F00397A9F028C081E48093760021309B
:100A700031F18FEF80937B0081E090E09093BA009A
:100A80008093B9001CC08AE518C08091D40015C0BD
:100A90008091D8008093760080917D00833479F432
:100AA000213069F482E090E090939300809392006B
:100AB00084E180937B0003C084E180937600909171
:100AC00076009FB980917B00E82FFF27DF01A458B3
:100AD000BF4F8091DB008C93E454FF4F90830E94C2
:100AE000060580917B008F5F80937B00843008F443
:100AF000A0CF0895B499FECF8FEF8FB980E590E035
:100B00000E94FF0410927B00779BFECF84E190E06F
:100B10000E94FF042FB12093DB0080917B00992776
:100B20008330910561F1843091054CF48130910559
:100B300009F18230910504F5892B69F036C08530C2
:100B4000910501F185309105ECF086309105D1F0E9
:100B50000797D1F02AC083E780937600213041F1D6
:100B600084E180937B0081E090E09093BA008093D1
:100B7000B9001EC08AE51AC08091D40017C08091C8
:100B8000D80014C080E812C080E88093760080917D
:100B90007D00833469F482E090E090939300809329
:100BA000920084E180937B0003C084E1809376000F
:100BB000909176009FB980917B00E82FFF27DF019D
:100BC000A458BF4F8091DB008C93E454FF4F908377
:100BD0000E94060580917B008F5F80937B00B49913
:100BE00003C0883008F490CF089580917B00992746
:100BF00084309105C1F08530910534F4823091053F
:100C000061F0039761F008958630910591F0863088
:100C100091052CF0079779F0089583E001C082E0F8
:100C20008093760008958091D2009091D300892B13
:100C300011F081E0F5CF109276000895089580912B
:100C40007B0099278430910509F18530910534F4B2
:100C50008230910561F0039751F008958630910537
:100C600089F08630910534F0079791F0089510923D
:100C70007600089580917F00882341F482E080937C
:100C80007600089580917F008823C9F381E0F7CF33
:100C900080917F00882311F48AE0F1CF84E1EFCFC7
:100CA00080917B0099278430910591F085309105E2
:100CB00034F48230910591F0039781F008958630E5
:100CC000910541F0863091054CF0079739F0089571
:100CD00082E001C081E08093760008951092760052
:100CE0000895089580917B00992784309105E1F063
:100CF0008530910534F482309105B1F00397A1F06D
:100D000008958630910581F0863091051CF0079793
:100D100059F0089580917F00882311F484E001C088
:100D200087E08093760008951092760008950895E4
:100D300080917B0099278430910519F185309105C8
:100D400034F48230910561F0039799F01DC086302C
:100D50009105B9F086309105A4F0079791F014C081
:100D60008091770090917800892B59F0109276004D
:100D70000BC08091770090917800892B11F081E071
:100D800001C08FEF8093760080917F00882359F413
:100D900080918000813039F481E090E09093780078
:100DA000809377000895109278001092770008954C
:100DB00008958091D2009091D3000097C1F4809162
:100DC0007B0099278430910599F18530910534F4A1
:100DD0008230910569F1039759F1089586309105A4
:100DE00039F18630910524F1079711F108950197A3
:100DF000029720F580917B00992784309105A1F01E
:100E00008530910534F48230910561F0039751F0FB
:100E100008958630910561F0863091054CF0079772
:100E200051F008958FEF01C083E08093760008951C
:100E30001092760008958AE58093760008950895CB
:100E400080917B0099278430910589F08530910548
:100E500034F48230910559F0039749F00AC0863086
:100E6000910529F08630910514F0079711F410923E
:100E7000760080917F008823D9F48091D2009091F0
:100E8000D3008130910549F0823091051CF4009720
:100E900021F00895029731F0089590939300809384
:100EA0009200089583E090E09093930080939200E5
:100EB0000895089580917B0099278430910589F0E9
:100EC0008530910534F48230910559F0039749F04B
:100ED0000AC08630910529F08630910514F00797F5
:100EE00011F41092760080917F00813039F481E016
:100EF00090E09093D3008093D2000895882321F44A
:100F00001092D3001092D2000895089580917B0032
:100F100099278430910591F08530910534F4823021
:100F2000910561F0039751F00FC08630910531F0C3
:100F3000863091051CF0079721F006C010927600CC
:100F400003C08AE58093760082E090E09093D3001E
:100F50008093D200089580917B0099278430910579
:100F600091F08530910534F48230910571F003974A
:100F700061F008958630910541F0863091052CF09E
:100F8000079731F0089582E004C01092760008952A
:100F90008AE58093760008950895B499FECF109263
:100FA0007B0080E590E00E94FF0480917B00883008
:100FB00008F092C0779BFECF84E190E00E94FF048E
:100FC0009FB19093DB0080917B00882381F483EFB5
:100FD00080937600913009F465C084E180937B00B2
:100FE00081E090E09093BA008093B9005BC08130BB
:100FF00011F48AE551C08250863008F050C08091CB
:101000007D0099278634910559F187349105A4F420
:1010100083349105A1F1843491053CF48034910529
:10102000B9F18134910541F136C08434910551F113
:101030008534910591F02FC08C349105B9F08D3431
:10104000910524F48734910571F025C08D34910504
:1010500081F08F349105C9F01EC00E94F50522C0B1
:101060000E941F061FC00E9450061CC00E947206EC
:1010700019C00E94980616C00E94D90613C00E948B
:10108000200710C00E945A070DC00E9486070AC0A0
:101090000E94AB0707C084E18093760003C084E11F
:1010A00080937B00909176009FB980917B00E82F20
:1010B000FF27DF01A458BF4F8091DB008C93E454DD
:1010C000FF4F90830E94060580917B008F5F809385
:1010D0007B00883008F46ECF80917D00843409F461
:1010E000000008950895B499FECF10927B0080E52A
:1010F00090E00E94FF0480917B00843108F059C089
:10110000779BFECF84E190E00E94FF048FB1809333
:10111000DB0080917B009927AA27BB27FC0144971D
:1011200058F5E65DFF4FEE0FFF1F0590F491E02D9F
:10113000099489E722C08AE520C08091D4001DC0AF
:101140008091D8001AC080E818C01092760017C0AD
:101150001092760080917D00833489F480917F0025
:10116000813069F482E090E0909393008093920044
:1011700084E180937B0003C084E1809376009091AA
:1011800076009FB980917B00E82FFF27DF01A458EC
:10119000BF4F8091DB008C93E454FF4F90830E94FB
:1011A000060580917B008F5F80937B00843108F47B
:0411B000A7CF089528
:1011B4005265762E0A0000050200000000000009B6
:0611C40001000000000024
:00000001FF
